:1000000019C05BC96BC42BC301C5C6C22EC03CC09E
:100010002CC02BC02AC091C59BC57CC5A3C925C0D7
:1000200024C023C022C021C020C08CC11EC01DC05E
:1000300038C81BC011241FBECFEFD4E0DEBFCDBF38
:1000400011E0A0E0B1E0E4ECFCE102C005900D920B
:10005000AA33B107D9F711E0AAE3B1E001C01D92BC
:10006000A03EB107E1F740D02CCECACF82E080930A
:10007000B00096E09093B1001092B2009DE790938B
:10008000B3008093700008951F920F920FB60F92E5
:1000900011248F939F9380913D018F5F80933D0149
:1000A00091E090933A01893179F410923D01909357
:1000B0003B0180913E018F5F80933E018A3021F4A5
:1000C00010923E0190933C019F918F910F900FBE33
:1000D0000F901F901895269A87B18C6087B92F9A38
:1000E00087E08BBB78940895CFEFD4E0DEBFCDBF1F
:1000F00005DCC3D13CDABADFEEDF53D1F0D46AD6E7
:1001000049DA80913A018823A9F010923A0118D473
:100110008091690181114AD180917501882319F07C
:1001200081508093750190E080910E01811191E0E2
:10013000892FF3D580913B01882371F010923B0108
:1001400091E0909373018091D701882329F0815029
:100150008093D7019093D60180913C01882311F0C0
:1001600010923C0180917301882309F47EC01092A3
:10017000730180910D01882309F077C020916401FB
:10018000409163016091570181EC78D629B146B165
:1001900063B180EC73D620916D0140916B01609149
:1001A0006A0183EC6BD620916201409161016091FC
:1001B000710184EC63D680917C018823F1F0109268
:1001C0007C0180912001880F880F880F20911F01EA
:1001D000220F220F282B90911301990F8091120169
:1001E000982B80910E018295807F892B282B40913E
:1001F0001E01609111018EEC41D68091680180FF53
:100200000BC08E7F8093680120915C0140915A0160
:1002100060915B0182EC32D68091680181FF0BC056
:100220008D7F8093680120915F0140915D01609115
:100230005E0187EC23D640916701442349F0415089
:1002400040936701209160016091600185EC16D6B2
:1002500040917801442321F020E060E089EF0ED640
:100260008091690181608093690180917201882386
:1002700061F0A2D5882349F06091720161506093CA
:10028000720120E040E08FEFF9D510DB29DC80918E
:100290000D01882309F435CFF894109268001DBA37
:1002A00010927A0025D468D97AD01DD167D2A2D114
:1002B00019D280E88093BC00909164008FEE809307
:1002C000640080E280936B0081E08BBB80916800CA
:1002D00081608093680083B7817F846083BF83B728
:1002E000816083BF7894889583B78E7F83BF909316
:1002F0006400C3D03CD9BADEEEDE53D0F0D36AD569
:1003000049D982E08093D70110920D01FACE9093E3
:10031000400180933F0108958FE880937A0008950B
:1003200010927A00089580937C00EAE7F0E08081E3
:1003300080648083089520917800822F2091790035
:10034000922F08951F920F920FB60F9211242F93A0
:100350003F934F935F936F937F938F939F93AF934D
:10036000BF93EF93FF93E0913F01F0914001099516
:10037000FF91EF91BF91AF919F918F917F916F917D
:100380005F914F913F912F910F900FBE0F901F9053
:100390001895809169018260809369010895C0DF9A
:1003A000089589EC91E0B3DFB7DF089580914101B2
:1003B000882339F4809169018E7F8093690186E0FA
:1003C0002EC0813099F5B7DF9C0188B18170809390
:1003D0005C012932310528F440990BC0409A389AC3
:1003E00008C083E0283E380720F0409B02C04098B8
:1003F000389820935A0130935B01809168018160A5
:1004000080936801809169018D7F8093690180915B
:100410006201882319F081E08093420187E083DF45
:10042000809141018F5F809341010895823021F5D1
:1004300080916201882319F081E0809342017BDF83
:1004400080935D0190935E0180914201882321F0A9
:1004500081E080935F0102C010925F01109242011F
:1004600080916801826080936801809169018D7F2D
:10047000809369011092410108953998419A8AB197
:100480008F738AB98BB1806C8BB984B1877E84B944
:1004900085B1886185B953985B9A8091D501813087
:1004A00019F4509A519A549A88E180936B00809184
:1004B000680081608093680082E080936C00809186
:1004C000680082608093680080E880936D0080916E
:1004D00068008460809368008091690088608093E0
:1004E0006900E99A08954198399A8BB18F738BB955
:1004F0008AB1806C8AB985B1877E85B984B18861FB
:1005000084B95B98539A0895823029F4609300016E
:100510006093020108958350823020F460930101BA
:10052000609303010895809162018B7F8093620143
:1005300010926A0180916F018E7F80936F018BB161
:100540008C7F8BB9089590916201946090936201C1
:1005500080936A0180916F0180FD03C088EC8093D5
:1005600045015998589A08954E9B04C04F9B02C06C
:1005700082E003C04F9903C081E0E5DF089582E087
:1005800080936A0108954F9B03C081E0DCDF0895EA
:1005900082E080936A0108951F920F920FB60F9226
:1005A00011248F934F9904C081E080930E0102C003
:1005B00010920E0180916F0180FD03C088EC809342
:1005C000450180916A01882369F0815080936A0116
:1005D000882341F48BB18C7F8BB95898599A86E067
:1005E0008093450184E08BBB8F910F900FBE0F90DD
:1005F0001F90189580916201877F8093620110920D
:100600006B0180916F018D7F80936F018BB18C7F27
:100610008BB90895909162019860909362018093E4
:100620006B0180916F0181FD03C088EC80934601CE
:100630005898599A08951B9902C0599B05C082E0A9
:10064000E9DF81E08093480108951C9902C0599B1D
:1006500005C082E0DFDF82E08093480108951F92A9
:100660000F920FB60F9211248F939F9383B1992706
:100670008095909588719070892B59F180916F01C8
:1006800081FD03C088EC8093460180916B01882333
:1006900001F1982F915090936B018091480188232C
:1006A00061F0813019F41B9908C004C0823029F42C
:1006B0001C9903C010926B0102C0992351F410924F
:1006C00048018BB18C7F8BB95998589A88E08093F8
:1006D000460181E08BBB9F918F910F900FBE0F90D1
:1006E0001F901895809162018F7E80936201109215
:1006F0006D0180916F018B7F80936F0180917001FC
:100700008E7F809370015C98289808959091620183
:1007100090619093620180936D01609302018091DA
:100720006F0182FD03C08AEF809347015C9890912E
:10073000700191609093700185B1892B85B90895FE
:100740008FEF80936C0165E082E0E0DF0895809197
:100750006101882321F465E081E0D8DF089582E01B
:1007600080936D01089580916101813019F465E0F5
:10077000CDDF089582E080936D010895809162013C
:100780008C7F809362011092710180916F01877F4D
:1007900080936F0180917001897F8093700185B192
:1007A000897F85B90895982F809162018160809337
:1007B00062019093710180914A01813039F44B9B21
:1007C00005C0992319F09F5F9093710110924A011F
:1007D00080916F0183FD03C08AEF8093490160938C
:1007E0000301909170019B7F92609093700185B19D
:1007F000892B85B90895982F80916201826080933A
:1008000062019093710180914A01882339F44B9BD6
:1008100005C0992319F09F5F9093710181E0809347
:100820004A0180916F0183FD03C08AEF80934901E3
:1008300060930301909170019D7F9460909370018B
:1008400085B1892B85B90895282F962F882369F4BF
:1008500040FF08C06093450180916F0181608093E3
:100860006F0160E0862F6FDE0895813069F440FFEC
:1008700008C06093460180916F01826080936F0190
:1008800060E0862FC7DE0895823081F440FD02C00B
:10089000862F08C06093470180916F018460809328
:1008A0006F0180E06091000131DF08958350823054
:1008B000A0F440FF07C06093490180916F018860F8
:1008C00080936F01233029F460910101892F6BDF40
:1008D000089560910101892F8EDF08951F920F9274
:1008E0000FB60F9211248F939F9380916F0183FD18
:1008F00003C08AEF80934901809171018823C9F078
:100900008150809371018823A1F490917001997FA7
:100910009093700185B1897F85B98AE08093490100
:1009200080914A01882311F4946001C092609093F1
:1009300070019F918F910F900FBE0F901F9018958F
:100940009091430180910201981709F428988091B1
:100950000301981719F485B1897F85B9892F8F5FB5
:1009600080934301863039F41092430185B1909110
:100970007001892B85B980916C01882361F08150C9
:1009800080936C01882339F4809170018E7F80936D
:1009900070015C98289880914701882341F081502C
:1009A00080934701882319F49DDE10920201809103
:1009B0004501882331F0815080934501882309F453
:1009C000B2DD80914601882331F081508093460149
:1009D000882309F40FDE80914901882331F081508A
:1009E00080934901882309F4C9DE8091440188235A
:1009F00061F0815080934401882339F482E08BBBFD
:100A00008091680082608093680008951F920F9221
:100A10000FB60F9211242F933F934F938F939F9371
:100A200082E080934401809168008D7F809368000C
:100A300031994BC08091610191E0892780936101D8
:100A400040916C01442329F180916D018130F1F4D2
:100A500080916E01882389F0242F332799274097AE
:100A60002817390754F4809161018E7F80936101CA
:100A700010926C0110926E010CC08AEF80934701B6
:100A800040936E018FEF80936C011FC08FEF8093B6
:100A90006C0180916F0182FD03C08AEF8093470152
:100AA00080916D01882389F0815080936D018823A6
:100AB00061F4809170018E7F809370015C9828981A
:100AC00028985C9A84E0809347019F918F914F9181
:100AD0003F912F910F900FBE0F901F90189591E0AE
:100AE000909380008AE08093810090936F00089536
:100AF00010928100EFE6F0E080818D7F8083429844
:100B000080914C01837F80934C0180818B7F808317
:100B1000439808951F920F920FB60F9211248F934E
:100B20009F9388B190914C01892B88B99F918F91A7
:100B30000F900FBE0F901F9018951F920F920FB637
:100B40000F92112442980F900FBE0F901F9018958E
:100B50001F920F920FB60F92112443980F900FBE61
:100B60000F901F901895582FE1E1F1E013C020FF7E
:100B700002C05E7F05C021FF03C05D7FEEE1F1E0B2
:100B800091E092834187662329F0608783858823DB
:100B900009F49487252F3327C90183709070892B1E
:100BA00031F70895582FE1E1F1E00BC020FF02C0BA
:100BB0005E7F05C021FF03C05D7FEEE1F1E067834A
:100BC0004683252F3327C90183709070892B71F7D5
:100BD0000895582FE1E1F1E00DC020FF02C05E7FD3
:100BE00005C021FF03C05D7FEEE1F1E06111648388
:100BF00041114583252F3327C90183709070892BBC
:100C000061F708950F931F93082F162F80911201FB
:100C10008823A1F480911301882381F480911F011E
:100C2000882361F480912001882341F44AE061E047
:100C300083E0CFDF412F602F83E095DF1F910F917D
:100C40000895482FE1E1F1E051E00EC020FF02C01D
:100C50004E7F05C021FF03C04D7FEEE1F1E06383CD
:100C60005183128213861486242F3327C90183707F
:100C70009070892B59F70895FC018181882329F10F
:100C800082858823F9F481E080937C01638120814F
:100C90003581822F9927462F5527261738F4830F41
:100CA000911D841795073CF4230F09C0831B9109FC
:100CB000481759071CF06083118207C0231B20834B
:100CC000848182878285815082878385882331F061
:100CD00081508387882311F481E084878181882370
:100CE000D9F484858823C1F080858F3F21F081501D
:100CF0008087882319F08185838701C012829681BD
:100D00008081981718F08781838301C0938381E0E5
:100D1000818384818287148608951F93182F809180
:100D20004D01811729F010934D0181E080937C01E2
:100D300081E191E0A1DF8EE191E09EDF2091110140
:100D4000263010F0112361F080914C018B7F80934D
:100D50004C0180916F008D7F80936F0042980AC094
:100D600080914C01846080934C0180916F0082607F
:100D700080936F0090911E01963010F0112361F066
:100D800080914C01877F80934C0180916F008B7F15
:100D900080936F0043980AC080914C0188608093D3
:100DA0004C0180916F00846080936F0020938800D5
:100DB00090938A001F910895E0913701F0913801D6
:100DC00020E030E093818481981711F421E030E035
:100DD000C9010895FCD08BE597E0EFD082EB97E056
:100DE000F1D0809137019091380116D20895E091A9
:100DF0003701F091380193818481981719F080E0D0
:100E000090E0089510D190E0813009F491E081E004
:100E10009827892F992708950F931F93CF93DF93D6
:100E2000AC01E0913701F091380123818481281BC6
:100E30003327828199270497821793073CF403C0D4
:100E400084E08093780180E090E013C0F894EA0198
:100E50008A010C5F1F4F6991809137019091380191
:100E6000ECD1882369F7C017D107A9F7789481E0FE
:100E700090E0DF91CF911F910F910895CF93DF9371
:100E8000CDB7DEB724970FB6F894DEBF0FBECDBF47
:100E900089836A834B832C83CE010196BDDF99271A
:100EA00087FD909524960FB6F894DEBF0FBECDBF98
:100EB000DF91CF9108950F931F93CF93DF938430E9
:100EC00011F085E00FC0E0913001F09131012381F4
:100ED0008481281B332782819927049782179307DF
:100EE00024F481E0809378010DC0EB018B010C5F4D
:100EF0001F4F699180913001909131019ED1C017AF
:100F0000D107B9F7DF91CF911F910F9108950F93FA
:100F10001F93CF93DF93BC01E0913001F091310139
:100F200093818481981739F403C082E0809378011B
:100F300080E090E012C0EB018B010C5F1F4FBE01FF
:100F4000809130019091310197D1882371F72196DA
:100F5000C017D107A1F781E090E0DF91CF911F91F9
:100F60000F9108950F931F93CF93DF93082FEB01F9
:100F7000E0913701F091380193818481981739F419
:100F800003C083E08093780180E090E011C010E01E
:100F90000BC0BE01610F711D809137019091380126
:100FA0006BD1882371F71F5F101799F781E090E0EC
:100FB000DF91CF911F910F910895909354018093E9
:100FC000530108959093560180935501089510920E
:100FD0004E01459A449A84E58093BA0080E6809356
:100FE000B90080E28093B80085EC8093BC0008953E
:100FF000FC0180914E01813019F48FEF9FEF08952D
:10100000F0935001E0934F0181E080934E01808185
:10101000880F809351011092520185EE8093BC009D
:1010200080E090E0089580914E0199270895CF9334
:10103000DF93CDB7DEB721970FB6F894DEBF0FBEB2
:10104000CDBF198203C089818F5F898389818F3FDA
:10105000D1F785EE8093BC0021960FB6F894DEBFE1
:101060000FBECDBFDF91CF910895FC0180914E015D
:10107000813019F48FEF90E00895F0935001E093E0
:101080004F0181E080934E018081880F8F5F8093B4
:1010900051011092520185EE8093BC0080E090E0F7
:1010A00008951F920F920FB60F9211242F933F9322
:1010B0004F935F936F937F938F939F93AF93BF9360
:1010C000EF93FF938091B9009927887F90708039C2
:1010D000910509F444C081399105E4F48037910504
:1010E000C1F18137910554F48036910591F188362C
:1010F000910579F1892B09F47BC07DC08038910579
:1011000071F18838910509F447C08837910509F0D5
:1011100072C01FC0803B910509F442C0813B91051C
:101120005CF4803A910559F1883A9105C9F1883902
:10113000910509F060C030C0803C910509F452C0AF
:10114000883C910509F44EC0883B910509F053C0D5
:101150003AC081E080934E011092C20147C0809155
:10116000C2019091BB00E82FFF27ED53FE4F908303
:101170008F5F8093C2018430C8F185E83AC08091C6
:10118000C201843039F4E0915301F091540163ECD1
:1011900071E0099510924E018091BC00856C29C0C8
:1011A00081E080934E01E0915501F0915601309716
:1011B00051F06EEB71E084E00995882321F01092E4
:1011C000BD0190E004C09091BD01943068F4E92F16
:1011D000FF27E254FE4F80818093BB009F5F909376
:1011E000BD0104C010924E011092BB0085EC01C0FD
:1011F00085ED8093BC00FF91EF91BF91AF919F91DE
:101200008F917F916F915F914F913F912F910F90AF
:101210000FBE0F901F901895FC0113821482089541
:10122000FC0120E030E083819481891B9281891741
:1012300011F421E030E0C9010895DC01FC012381B3
:1012400092818481F22FF81BF91719F481E090E064
:101250000895E22FFF27892F99270197E823F92383
:101260008D919C911197E80FF91F60832F5FFD010D
:10127000238380E090E00895CF93DF93DC01EC01BD
:101280002C818B81281719F482E090E013C0E22FA3
:10129000FF27ED018A8199270197E823F9238D9192
:1012A0009C91E80FF91F8081FB0180832F5F2C83C5
:1012B00080E090E0DF91CF9108951F920F920FB6DA
:1012C0000F9211248F939F938091CD0183FF04C0CF
:1012D00080E88093CC013FC08091CD0184FF1EC087
:1012E00085B58E7F85BD8091CC018095982F969590
:1012F000880F891B8093CB018091CD018F7E8093D5
:10130000CD018091CD0180628093CD018CE08093EE
:10131000CA011092CF011092CE011DC08091CD0163
:1013200085FF0EC08091CB018093CC0185B5816093
:1013300085BD8091CD018F7B8093CD01E8980BC056
:101340008FEF8093CC0185B5816085BD8091CD0103
:1013500080618093CD019F918F910F900FBE0F9070
:101360001F9018951F920F920FB60F9211242F9372
:101370003F934F938F939F935D988091CC018823E7
:1013800021F08091CC01815013C08091CD0180FF6C
:1013900086C08091CD0186FF0EC08091CD0188600E
:1013A0008093CD018091CD018F798093CD0180E82C
:1013B0008093CC01D2C08091CD0185FF63C0809124
:1013C000CA0181508093CA014A9B13C08091CE010B
:1013D0009091CF014091CA0121E030E002C0220F7C
:1013E000331F4A95E2F7822B932B9093CF01809382
:1013F000CE018091CA018823A9F582E0809367011C
:101400008091CD0188608093CD018091CD018F7D49
:101410008093CD0180E88093CC018091CE019091A2
:10142000CF018F73809360018091CE019091CF01A5
:10143000807C97708054974029F480916001806887
:10144000809360018091CE019091CF0193FF04C001
:1014500080916001806403C0809160018F7B8093E4
:10146000600108C08091CD0180648093CD0180E847
:101470008093CC0180916900816080936900E09A3B
:10148000E89A6BC08091CD0183FF67C08091CD0148
:10149000877F8093CD0185B58E7F85BD5EC08091AD
:1014A000CD0182FF0AC08091CD0192E0892780930F
:1014B000CD018091CD018B7F26C08091CA01882308
:1014C00049F18091CA0181508093CA012091C701DE
:1014D0003091C8014091CA0181E090E002C0880FBC
:1014E000991F4A95E2F728233923232B21F4809171
:1014F000CD01826003C08091CD018D7F8093CD01AD
:101500008091CD0184608093CD018091CB01809347
:10151000CC0119C08091CD0188608093CD0180916C
:10152000CD0181608093CD018091CD018D7F80932D
:10153000CD0180E88093CC01809169008160809327
:101540006900E09AE89A8091CD0181FF03C084B5DB
:10155000806202C084B58F7D84BD9F918F914F9131
:101560003F912F910F900FBE0F901F9018955D988F
:10157000559A08955D9A08955D98089583E084BD15
:1015800088E085BD16BC88BD83ED87BD82E0809371
:101590006E000895F3DF81E08093CD018091CD014D
:1015A00088608093CD0180E88093CC0185B581600F
:1015B00085BDE9E6F0E0808181608083E09AE89A69
:1015C000089585B58E7F85BDE898089585B58E7F91
:1015D00085BDE8980895EF92FF920F931F93082F0F
:1015E000E62E85B58E7F85BDE898C8DF1092CD01C7
:1015F0008EE08093CA011092CC011092CD01006C54
:1016000011271093C8010093C7018091C7019091E1
:10161000C80126E0880F991F2A95E1F79093C80129
:101620008093C7018091C7019091C801FF242FE3E7
:10163000E222FF248E299F299093C8018093C7013D
:1016400082E28093CB0185B5816085BD1F910F91AA
:10165000FF90EF900895CF93DF93CDB7DEB72C972F
:101660000FB6F894DEBF0FBECDBFFC018081803F76
:1016700009F056C0DF011196818183FF07C0809178
:10168000570183FD03C081E0809306018C9180FFA8
:1016900007C08091570180FD03C081E0809307015E
:1016A0008C9181FF07C08091570181FD03C081E0CB
:1016B000809308018C9184FF07C08091570184FDBD
:1016C00003C081E0809309018C9182FD07C0809165
:1016D000570182FF03C081E080930A018C9185FF4E
:1016E0000CC08091570185FD11C081E080930F01EE
:1016F000109210018C9185FD09C08091570185FFE2
:1017000005C010920F0181E0809310018C918093AD
:101710005701828180936301838180936401BDC0FE
:101720008F3721F4818180937201B7C0803911F025
:10173000823911F4CF011CC0873B21F481E08093F2
:101740000D01ABC08230B1F480EF9DE1DE01119656
:10175000FC010196E491ED932DE18C3F9207C1F7D6
:10176000CE01019659DBCE01059656DBCE010996D6
:1017700053DB93C08E3349F4E5E0F1E0119281E050
:10178000EE30F80709F489C0F9CF803D29F4438190
:10179000628181811EDA81C0813D21F46281818173
:1017A00050DA7BC0813921F46281818114DF75C0F8
:1017B000813821F462818181A7D66FC0823D29F4EE
:1017C000438162818181EED968C0843D29F44381DF
:1017D0006281818139D85EC0833D29F44381628171
:1017E0008181C1D957C08A3111F46FEF03C08B31A9
:1017F00021F460E083E025DA4DC08A3921F462816A
:10180000818100DA47C0803419F481819CD642C0BE
:10181000823311F488D63EC0833311F4A5D63AC082
:10182000883311F4B0D636C0813419F48181F2D6F0
:1018300031C0843311F4FFD62DC0853311F405D7A0
:1018400029C0863311F4D6D625C0803821F46281B0
:1018500081815CD71FC0893311F479D71BC08A33CB
:1018600011F481D717C0813311F46AD713C08033C4
:1018700011F438D70FC0823821F46281818193D767
:1018800009C0833821F462818181B5D703C08733D1
:1018900021F474D781E0809373012C960FB6F894ED
:1018A000DEBF0FBECDBFDF91CF9108950F931F9381
:1018B000CF93DF93CDB7DEB724970FB6F894DEBF92
:1018C0000FBECDBF8E010F5F1F4FC80120DB8823E5
:1018D00011F0C801C0DE24960FB6F894DEBF0FBE2B
:1018E000CDBFDF91CF911F910F91089583E0E2ED7D
:1018F000F1E0AFEBB0E0182ED3D1089583E0E2ED34
:10190000F1E0AFEBB0E0182EC6D1AFEFB1E0BBD144
:10191000802D8093D5010895A091DD01B091DE0165
:101920009D012F5F3F4F3093DE012093DD01ABD14E
:10193000802D8093D801E9EDF1E0D9012F5F3F4F71
:10194000A2D1802D819381E0ED3DF807B1F730936E
:10195000DE012093DD010895AC01DC0194D1802DDE
:101960008093D7015093DE014093DD01D5DF81E004
:101970008093D601089580910501882351F010923B
:10198000050180E090E0E8DF80915A0180937401C6
:10199000089580910601882329F0109206018FE1B5
:1019A00090E042C080910701882329F0109207013E
:1019B0008FE290E039C080910801882329F01092CD
:1019C00008018FE390E030C080910901882329F05D
:1019D000109209018FE490E027C080910A018823CA
:1019E00029F010920A018FE590E01EC080910F014E
:1019F000882329F010920F018FE690E015C08091A6
:101A00001001882329F0109210018FE790E00CC09C
:101A100090910C01903F51F481EF80930C0183E091
:101A200080930B018FE890E097DF0895903E51F48A
:101A300081EE80930C018FE990E08EDF85E080934A
:101A40000B010895903D31F48FEA90E085DF10920C
:101A50000C010895809176018823D1F080910B01CB
:101A6000882381F0913F21F46091740188E003C0E4
:101A7000609174018CE0AFDD80910B018150809307
:101A80000B0104C06091740184E0A5DD1092760121
:101A90000895FF920F931F9315C0FF240F2D112758
:101AA000C80187529E4FD7DD08521E4FF801818131
:101AB0008295869586958370F394F80EF3E0FF1572
:101AC00068F72ADF9091D8018091D701981710F01C
:101AD0009F3F19F71092D6011F910F91FF90089523
:101AE0001F938091D6018111D4DF8091D701882383
:101AF00009F441DF8091570182FF03C03FD6109265
:101B000071019091600180917701981709F4B9C033
:101B10008091600187FFB5C0109160011F738091B3
:101B2000600180916001809377018091D2018823C8
:101B300019F064E082E066D880917A01882369F028
:101B4000163159F480914B01882321F481E0809370
:101B50004B0109C010924B0106C01C3321F481E0F7
:101B600080937A0102C010927A0180914B01882300
:101B700009F487C01332E9F11432A0F41D3009F4DE
:101B800053C01E3030F41A3048F11C3009F079C0CF
:101B900035C0103209F451C0123219F1103109F078
:101BA00070C04FC0123309F451C0133340F41532E2
:101BB00089F1153248F1163209F063C016C01633A8
:101BC00079F1173320F4143309F05BC045C01833A2
:101BD00009F44AC0193309F054C04CC010933901BC
:101BE00050C080913901AFD44CC08091390112D5D9
:101BF00048C065E08091390189D543C020E040E0CC
:101C000061E087EB3BD93DC06091030180913901D0
:101C1000CAD537C06091030180913901ECD531C03C
:101C2000ADD560D5E7D42DC090E08091D201882356
:101C300009F491E09093D20124C040E061E082E099
:101C400003C040E061E081E08ED71BC080910301BA
:101C50008823B9F0815005C080910301853088F454
:101C60008F5F809303010DC080910201882349F0AA
:101C7000815005C080910201853018F48F5F8093F8
:101C800002011F910895F999FECFB2BDA1BDF89A46
:101C9000119600B40895F7DF01921A94E1F70895C0
:101CA000019003D01A94E1F70895F999FECFB2BDDF
:101CB000A1BD00BC11960FB6F894FA9AF99A0FBE1E
:041CC0000895FFCFB5
:101CC40005050505FF0100000000000000000000FC
:101CD4000000000000010200FF00000000000000FE
:101CE4000000010200FF00000000009D0120000030
:0A1CF4002B017D01200000320101E8
:0C1DF000C8000901C9790901CA000000FF
:00000001FF
